:020000040000FA
:1000000018308A00A22D0000FF00030E8301A1001A
:100010000A08A0008A010408A2007708A300780853
:10002000A4007908A5007A08A6007B08A70083131E
:1000300083128C308400001C1F280C1832282208E0
:1000400084002308F7002408F8002508F900260892
:10005000FA002708FB0020088A00210E8300FF0E0B
:100060007F0E09008A110A1241280A108A100A110B
:10007000820700340034103430348A3400340034C1
:100080002D34061D452806114628061564000C105F
:100090008A110A121F28871087162130F700F70BE4
:1000A0004F2800348C1A5628640052288C1E56287B
:1000B0001A088316D4008312981C64281A08831621
:1000C000D40083121812181683165408F8008312ED
:1000D00000342908073C031D722807300C1E6E28C7
:1000E0009900B12805308316C2004208063C031966
:1000F000B0284208053C031DAA282930C4008312F9
:100100006F088316C100043083120C1E85289900E5
:100110006F080C1E892899008316C30183126F088B
:10012000831643020318A428440884000008C5006D
:1001300083120C1E99289900831644088400000835
:10014000C106C40AC30A8E28410883120C1EA628C1
:10015000990083168312522078088316C2007528EE
:10016000831200349030A9000130AA003930AB006E
:10017000831681138312861DC0280230AC00C2286A
:100180000130AC000430EF0069200034E03084001E
:1001900000080319D8280630F800F701F70BCE281D
:1001A000F80BCD287B30F700F70BD428800BCB2839
:1001B00000349130A9000230EF0069202A08F700CE
:1001C000F7080319F828013077020319FE280230D6
:1001D0007702031904290330770203190A2906302C
:1001E00077020319102907307702031916291D29F0
:1001F000813083169900263098001F2940308316DD
:100200009900263098001F29203083169900263047
:1002100098001F29153083169900263098001F2951
:100220000A3083169900263098001F29043083165F
:100230009900263098001F29831283161F29023047
:10024000E0008312C6208A110A16AD28F701F801D2
:100250008316540803105518F707F70CF80CD51837
:10026000F707F70CF80C5519F707F70CF80CD51928
:10027000F707F70CF80C551AF707F70CF80CD51A16
:10028000F707F70CF80C551BF707F70CF80CD51B04
:10029000F707F70CF80C831200349230A9006F08AE
:1002A000413C03196C290130AA008316BA013A08AF
:1002B0003F3C031C6A2902303A07293E84003A0871
:1002C000D4000530D50083122621780880008316DB
:1002D000BA0A5729A32983128316BA013A083F3C68
:1002E000031C852901303A07293E84000008BC0020
:1002F0003A08D4000530D5008312262178088316E9
:100300003C02031D8529BA0A6E293A083F3C031CAA
:100310008B2901308C2900308312AA008316BA0180
:100320003A083F3C031CA32902303A07293E8400C7
:100330003A08D4000530D5008312262178088000C1
:100340008316BA0A902942308312EF0069208A117D
:100350000A16B5289530A9000508AA000608AB00C2
:100360000708AC00053083169F0083121F08383938
:10037000C1389F000030F8001F08C73978049F007B
:10038000A630F700F70BC22900001F151F19C62958
:100390001E08AD000830F8001F08C73978049F0018
:1003A000A630F700F70BD22900001F151F19D62918
:1003B0001E08AE000630EF00692000346F08073CCD
:1003C000031DF5292A088316850083122B0883163E
:1003D000860083122C088316870083122D0885005F
:1003E0002E0886002F088700AA218A110A16BD2828
:1003F0002A088316BB002B30BC00BA0102308312DE
:100400006F0283163A020318312A3B08BB0ABD006B
:100410003C08BC0A84000008BE003D088312031794
:100420008D008F01831603133E08831203178C007F
:1004300083168C130C15831203130B08F7008B1310
:100440008316031755308D00AA308D008C148C183C
:10045000272A0C117708831203138B048316BA0A18
:10046000FE2907308312A9000130EF0069208A11AC
:100470000A16CD282A088316BB002B30BC00831235
:100480002B08EF008316BA0183126F0883163A0215
:1004900003185E2A3C08BC0A84003B08BB0ABE0065
:1004A000831203178D008F0183168C130C14831293
:1004B0000C08800083160313BA0A442AE33083121F
:1004C000A9000230EF0769208A110A16D528E53005
:1004D000A9000130AA000230EF0069208A110A1633
:1004E000DD28E730A9004630AA000230EF0069207D
:1004F0008A110A16E5288712003480308316870592
:1005000081308704D93086050616DB3085051B301F
:1005100085040515851686148312871107124B2052
:100520007B2287142130F700F70B942A4B207B2283
:1005300087142130F700F70B9B2A0034831622081A
:100540001F3C031DC22AE2016208053C031CC12AAC
:100550008312871503108316E00C0318B32A831245
:100560000712B52A8316831207162130F700F70BFE
:10057000B72A87112130F700F70BBC2A8316E20A4D
:10058000A42AF62B6008E03E0318F62B203E8312C7
:10059000FD2B071287158711071287158711071280
:1005A000871587110712871587110712871587117D
:1005B0000712871587118316F62B071687158711E3
:1005C00007128715871107128715871107128715DC
:1005D0008711071287158711071287158711831650
:1005E000F62B071287158711071687158711071233
:1005F000871587110712871587110712871587112D
:100600000712871587118316F62B07168715871192
:100610000716871587110712871587110712871587
:1006200087110712871587110712871587118316FF
:10063000F62B0712871587110712871587110716E2
:1006400087158711071287158711071287158711DC
:100650000712871587118316F62B07168715871142
:100660000712871587110716871587110712871537
:1006700087110712871587110712871587118316AF
:10068000F62B07128715871107168715871107168E
:10069000871587110712871587110712871587118C
:1006A0000712871587118316F62B071687158711F2
:1006B00007168715871107168715871107128715E3
:1006C000871107128715871107128715871183165F
:1006D000F62B071287158711071287158711071246
:1006E0008715871107168715871107128715871138
:1006F0000712871587118316F62B071687158711A2
:100700000712871587110712871587110716871596
:10071000871107128715871107128715871183160E
:10072000F62B0716871587110716871587110712ED
:1007300087158711071687158711071287158711E7
:100740000712871587118316F62B07128715871155
:10075000071687158711071687158711071687153E
:1007600087110712871587110712871587118316BE
:10077000F62B071687158711071687158711071699
:100780008715871107128715871107168715871197
:100790000712871587118316F62B07128715871105
:1007A00007128715871107128715871107168715F6
:1007B000871107168715871107128715871183166A
:1007C000F62B071687158711071687158711071649
:1007D0008715871107168715871107168715871143
:1007E0000712871587118316F62B83160000000069
:1007F000000000000000831200340A108A100A155D
:100800008207C92ADD2AF12A052B192B2D2B412B12
:10081000552B692B7D2BF52B912BF52BF52BA52B30
:10082000F52BF52BF52BF52BF52BF52BF52BF52BC8
:10083000B92BCD2BF52BF52BF52BF52BF52BF52B1C
:10084000E12B01308316AA000230A500A300A60107
:100850002608A4000830A8000E30A9006430A700C4
:100860000930B8000630E00083129E22003483165F
:10087000A5012508A3006430A600A4000830A80044
:100880000E30A9001930B3006430B4000330B50055
:100890001F305F02FF3E0318582C013E83125C2C70
:1008A00064308316E0008312C6208316582C83160A
:1008B00083128A110A124B2E0A108A100A15820717
:1008C000502C7D222808FF3E03184E2E013E4F2E4D
:1008D00083165D08DE00A101A0015E08A200A90147
:1008E000A701AA012030AC00AB01AE000730AD007B
:1008F0000130AF00B0010130B100B201B6013710D4
:10090000B8012208F7001030220283120319E52CE7
:10091000123077020319F02C153077020319FE2CE0
:100920001130770203190A2D133077020319152DA0
:10093000163077020319252D1C3077020319312D4B
:100940001730770203193D2D1D3077020319492D09
:10095000183077020319552D193077020319602DCD
:100960001A30770203196C2D143077020319782D91
:10097000043077020319902D1B3077020319A82D3C
:10098000033077020319C02D073077020319CB2DEE
:100990000B3077020319D72D0C3077020319E32DA2
:1009A000083077020319EF2D093077020319012E61
:1009B000053077020319132E0630770203191F2E14
:1009C0000A3077020319332E462E08308316A5000D
:1009D000A300A6012608A4000830A800B8014C2EE8
:1009E00008308316A500A300A6012608A40008303D
:1009F000A8000130B6000130B8004C2E0D3083162F
:100A0000A500A300A6012608A4000830A800033012
:100A1000B8004C2E04308316A500A300A6012608BA
:100A2000A4001830A800B8014C2E02308316A5008F
:100A3000A300A6012608A4001830A8001730A900BA
:100A40000130B6000130B8004C2E08308316A500E6
:100A5000A300A6012608A4001830A8000330B8009F
:100A60004C2E03308316A300A4010630A500A60176
:100A70000830A8000430B8004C2E08308316A500BA
:100A8000A300A6012608A4000830A8000530B8007D
:100A90004C2E08308316A500A300A6012608A4004A
:100AA0000830A8000830B8004C2E14308316A5007A
:100AB000A300A6012608A4000830A800B8014C2E07
:100AC00008308316A500A300A6012608A40008305C
:100AD000A8000330B8004C2E04308316A500A300F4
:100AE000A6012608A4001830A8000330B8004C2E38
:100AF00001308316A500A300A6012608A400083033
:100B0000A8000E30A9000230AF000130B000023062
:100B1000B1000130B2000330B6000230B8004C2EF4
:100B200002308316A500A300A6012608A4001830F1
:100B3000A8001730A9000430AF000330B000043023
:100B4000B1000330B2000330B6000630B8004C2EBE
:100B500001308316A500A300A6012608A4001830C2
:100B6000A8001730A9000430AF000330B0000430F3
:100B7000B1000330B2000330B6000730B8004C2E8D
:100B800001308316AC00AB01AE00FF30AD00831224
:100B9000212483164C2E02308316AC00AB010330A7
:100BA000AE00FF30AD008312212483164C2E02309C
:100BB0008316AC00AB010330AE00FF30AD008312F2
:100BC000212483164C2E04308316AC00AB01073071
:100BD000AE00FF30AD008312212483164C2E03306B
:100BE0008316A300A4010630A500A6010830A800C2
:100BF0000430AF000330B0000330B6000430B8005A
:100C00004C2E03308316A300A4010630A500A601D4
:100C10000830A8000830AF000730B0000330B6003D
:100C20000430B8004C2E02308316AC00AB01033008
:100C3000AE00FF30AD008312212483164C2E083005
:100C40008316AC00AB010F30AE00FF30AD000430B6
:100C5000AF000330B0000430B1000330B2008312A3
:100C6000212483164C2E02308316A500A300A60172
:100C70002608A4001830A8000E30A9006430A70090
:100C80000330B6000230B8004C2E831283165E0883
:100C9000DF008312372C831683124E2E00340A1085
:100CA0008A140A158207682C2A088316BA003A08A3
:100CB000E0398312A80083163A08DD00831261240C
:100CC0000730A9000130EF0069208A110A16ED28CB
:100CD00083163A1083122A080139003A0319772E35
:100CE0006F08023C031D772E83163A1483120030DE
:100CF00083163A180130BB00BC0083124B20071149
:100D00000C3097000030F8000438920077308316DA
:100D10009200BC080319942E3C30831295001708EA
:100D2000CF3997009A2E831620308312950017082A
:100D3000CF3997004B2004308316BB00AF30E00062
:100D40008312C6208316BB0B9E2E07308312A90088
:100D50000130EF0069208A110A16F5280711970162
:100D600097014B200730A9000130EF0069208A115C
:100D70000A16FD28831622081F3C031DF92E831234
:100D8000871507162130F700F70BC42E8711213085
:100D9000F700F70BC92E8316E20162080D3C031C15
:100DA000EB2E8312871503108316E10CE00C031859
:100DB000DD2E83120712DF2E8316831207162130D1
:100DC000F700F70BE12E87112130F700F70BE62E25
:100DD0008316E20ACD2E8312871507162130F700FD
:100DE000F70BF02E87112130F700F70BF52E192F96
:100DF000831683128715071687118316E20162088E
:100E00000D3C031C152F8312871503108316E10C6C
:100E1000E00C03180F2F83120712112F8316831271
:100E2000071687118316E20AFF2E8312871507160D
:100E300087110330F700F70B1B2F64000034831673
:100E40005D08E00083129E2283165F08E1005E08C1
:100E5000E0008312BA26003483162A080139003ACA
:100E60000319422F2D085B02031D422F2E085C023E
:100E7000031D422F83127D2283165C08A1005B08AC
:100E8000A000792F5C082102031C4C2F031D542F56
:100E900020085B02031C542F5C081F3C0318792FA9
:100EA00021081F3C031C792F5C081F3C031C672F83
:100EB0002208DD008312612402308316DD003F30FA
:100EC000DF00FF30DE0083121F27782F83162208F1
:100ED000DD00831261248316DD013F30DF00FF3027
:100EE000DE0083121F2720308316A100A001831289
:100EF000831621085C02031C8C2F031D832F5B08C3
:100F0000200203188C2F0630E00083129E228316E5
:100F1000A00A0319A10A792F8312003483163C0812
:100F2000FD3E0318AF2F033E8312CB2F09308316EB
:100F3000BC002030DC00DB0183122C278316AF2F8E
:100F40000B308316BC00AF2F1F308316BC0020303F
:100F5000DC00DB0183122C278316AF2F83163C089D
:100F6000E00083129E2204308316E0008312C62024
:100F700083163C081F3C0319C72F0830E00083127A
:100F80009E2202308316E0008312C620831683124D
:100F90008A150A12942C0A148A140A158207962FAD
:100FA000A02FA42F8316C801470848020318F62F64
:100FB0004508FA004408C40A0319C50AC9007A089A
:100FC000CA00DC004908DB0083122C27831648087E
:100FD0004607C9000430D9004908DA008A1583128F
:100FE00045208A1102308316C807D42F831200349B
:100FF00000308C1A0130F8000034FF3FFF3FFF3F04
:1010000083163C08FD3E03183A28033E83123E280F
:101010008316E0018A1183129E228A153F308316BF
:10102000E100FF30E0008A118312BA268A150930E8
:101030008316E0008A1183129E228A1506308316D9
:10104000E0008A118312C6208A158316BC08031992
:101050003A280B308316E0008A1183129E228A15EB
:1010600006308316E0008A118312C6208A15831683
:101070003A28831683128A150A122E2D0A108A1016
:101080000A11820708282928082883165908E00031
:101090008A1183129E228A15831607165A08DB00CE
:1010A00022081F3C031D7628DC015C080F3C031C52
:1010B0007528831287150000071A6028031061281D
:1010C000031483165B088400840A800C8403800C5C
:1010D0002130F700F70B6A28831287112130F700BF
:1010E000F70B70288316DC0A55288F28DC015C0872
:1010F0000F3C031C8F28831287150000071A8228D3
:1011000003108328031483165B088400840A800C70
:101110008403800C831287118316DC0A77285B080E
:101120008400013084070310800C8403800C5B086A
:1011300084000008F700840A00083F39FA007708A5
:1011400084038000840A7A08800084030330F70057
:10115000F70BA8286400071283120034E7308400DC
:1011600000080319B828B62800000000800BB42836
:10117000003483162808E0008A1183129E228A1503
:1011800083162308E0008A118312C6208A1583166D
:101190002408E7008312AE208316A9080319D72874
:1011A0002908E0008A1183129E228A1583162708D7
:1011B000E7008312AE200034B920013083162007E7
:1011C000D6002108D7000318D70A5708DC005608B4
:1011D000DB008A1183122C278A15003483165008ED
:1011E0000739D5002208123C031D2429F830D00508
:1011F0003F30D105D4015508540203182429510861
:10120000FA005008D00A0319D10AD9007A08DA0086
:10121000DC005908DB008A1183122C278A15043060
:101220008316D900D630DA008312452002308316A7
:10123000DD005708DF005608DE008A1183121F27E1
:101240008A158316D40AFB28D401530854020318C4
:1012500051295108FA005008D00A0319D10AD900BF
:101260007A08DA00DC005908DB008A1183122C2787
:101270008A1583165208D20AD20A8400840A00080A
:10128000DA0084030008D9000230DD005A08DF00CC
:101290005908DE008A1183121F278A158316D40A83
:1012A00025292208123C031D892951081F3C0318D7
:1012B0005C290430D8005E290830D8005508D307CF
:1012C00058085302031889295108FA005008D00A17
:1012D0000319D10AD9007A08DA00DC005908DB00CA
:1012E0008A1183122C278A1504308316D900D63030
:1012F000DA008312452002308316DD005708DF0034
:101300005608DE008A1183121F278A158316D30A16
:101310006029831200348316D5010130540255022E
:101320000318B9295308D30AD30A8400840A000891
:10133000D70084030008D6000230DD005708DF0024
:101340005608DE008A1183121F278A150130831682
:101350002007D6002108D7000318D70A5708DC0059
:101360005608DB008A1183122C278A158316D50AAA
:101370008D2953088400840A0008D70084030008DC
:10138000D6000230DD005708DF005608DE008A1163
:1013900083121F278A15DC20003483163608FB3E93
:1013A0000318902B053E8312922B83164608CA0021
:1013B0004508C9004708CB004808CC004B08CE00C0
:1013C0004A08DC004908DB008A1183122C278A15A1
:1013D0008316CD014C084D0203180A2A01304D072F
:1013E0004E0784000008D0004E084D078400000816
:1013F000D1005008D2000230DD005008DF00510853
:10140000DE008A1183121F278A15DC200230831622
:10141000CD07EA29902B83164608CA004508C90063
:101420004708CB004808CC004B08CF000310CC0C79
:1014300049080739F7004A080039FA007708083CDC
:10144000CE004C020318262A4C08CE004A081F3C46
:1014500003186D2AFF3A031D312A4908033C03187B
:101460006D2ACD014C084D0203186C2A4A08FA0077
:101470004908C90A0319CA0AD0007A08D100DC0059
:101480005008DB008A1183122C278A1583164F0817
:10149000CF0ACF0A8400840A0008D1008403000820
:1014A000D0000230DD005108DF005008DE008A1154
:1014B00083121F278A1508308316E0008A118312D1
:1014C0009E228A1506308316E0008A118312C620F8
:1014D0008A158316CD0A322AA62A4A08D10049085D
:1014E000D0004B08D2004E08D3008312EE20DC203F
:1014F00083164E08CC0203104E0DF700CF070830BC
:10150000CD004D084C02031C962A2108D10020086A
:10151000D0004F08D2000830D3008312EE20DC2028
:1015200010308316CF070830CD07812A0730CC054D
:101530000319A62A2108D1002008D0004F08D200A4
:101540004C08D3008312EE20DC208316902B8316E8
:101550004608CA004508C9004708CB004808CC0027
:101560004B08D0000310CC0C4A081F3C0318BD2ABE
:101570003108D1003208D200C12A2F08D10030082A
:10158000D20049085205CF004A08DC004908DB00B8
:101590008A1183122C278A158316CF080319E52A8E
:1015A0004F085102CE004C020318D82A4C08CE0036
:1015B0005008D3004E08D40083128B2183164E08A6
:1015C000CC0203104E0DF700D0074C085205CD0099
:1015D0005208FF3ACC05CC080319FC2A5008D30066
:1015E0005108D40083128B2103108316510DF7008C
:1015F000D0075108CC02EB2ACD080319062B50085E
:10160000D3004D08D40083128B218316902B8316B0
:101610004608CA004508C9004708CB004808CC0066
:101620004B08CD000310CC0CCC0803198E2B4A08B4
:10163000FA004908C90A0319CA0AD3007A08D40073
:10164000DC005308DB008A1183122C278A158316CD
:101650004D08CD0ACD0A8400840A0008FA008403EC
:101660000008CE007A08CF004A081F3C0318422B1E
:10167000FF3A031D3F2B4908073C0318422B34084F
:10168000D2007A2B3308D2000230DD004F08DF0091
:101690004E08DE008A1183121F278A15B9200430F4
:1016A0008316D900D030DA00831245208316D20386
:1016B0000319622B4E085002031D442B4F085102A0
:1016C000031D442B4E085002031D792B4F08510275
:1016D000031D792B52083302D3003508D400530878
:1016E000D5008A11831226218A1578088316D20024
:1016F0007A2B8E2B5208D203003A03198C2B02301E
:10170000DD004F08DF004E08DE008A1183121F271C
:101710008A15B92083167A2BCC03142B902B8316B1
:10172000831200340A148A140A118207D5290B2A5D
:101730008F2BA72A072B83163C08FD3E0318E22BAC
:10174000033E8312E62B20308316C5000730C40009
:10175000C030C6000230C7008A118312D2278A1512
:1017600009308316E0008A1183129E228A15083000
:101770008316E0008A118312C6208A15FF30831673
:10178000C0040F30C1042030C6000730C500C0308F
:10179000C7000230C8008312CD218316BC0803198C
:1017A000E22B0B308316E0008A1183129E228A15E9
:1017B00008308316E0008A118312C6208A1583162A
:1017C000E22B831683128A150A12352D0A148A1405
:1017D0000A118207A32BD12BA32B83163C08FD3EB5
:1017E0000318112C033E83121A2C20308316DC00C0
:1017F0000930DB008A1183122C278A1509308316E1
:10180000E0008A1183129E228A158316112C0B3058
:101810008316E0008A1183129E228A158316112CEA
:1018200083160630E0008A118312C6208A158A15B5
:101830000A123F2E0A108A100A158207FE2B072C67
:10184000F52B83163808F63E0318682E0A3E8312DD
:101850006C2E83163B08BC003C08F700F708831287
:101860000319372C0130770203193B2C402C02302E
:101870008316BC00422C03308316BC00422C83121A
:101880008316BC013C08E0008A1183129E228A154F
:101890003F308316E100FF30E0008A118312BA2640
:1018A0008A158316BC08031D632CBD013D08063C48
:1018B000031C632C0630E0008A1183129E228A15D5
:1018C0008316BD0A562C0130E0008A1183129E2235
:1018D0008A1507308316E0008A1183129E228A152A
:1018E00008308316E0008A1183129E228A15083080
:1018F0008316E0008A118312C6208A1501308316F0
:10190000E0008A1183129E228A1507308316E000B8
:101910008A1183129E228A158316682E83163B082D
:10192000BC008A1183128E2F8A158316682E2030F0
:101930008316DC00DB018A1183122C278A150930FB
:101940008316E0008A1183129E228A151E308316A8
:10195000E0008A118312C6208A158316682E83162A
:101960003B08BC003C08F700F70883120319BD2CA4
:10197000013077020319C12CC62C09308316BE0032
:10198000C72C0B308316BE00C72C83128316E001D0
:101990008A1183129E228A153F308316E100FF30A0
:1019A000E0008A118312BA268A158316BD013D080C
:1019B000063C031CE42C0630E0008A1183129E22B0
:1019C0008A158316BD0AD72C3C08023C0319FE2C4D
:1019D0003E08E0008A1183129E228A151830831671
:1019E000E0008A1183129E228A1505308316E000DA
:1019F0008A118312C6208A15272D83160130E00034
:101A00008A1183129E228A1507308316E0008A11FC
:101A100083129E228A1508308316E0008A118312F1
:101A20009E228A150D308316E0008A118312C6208B
:101A30008A1501308316E0008A1183129E228A15CE
:101A400007308316E0008A1183129E228A158316BE
:101A5000682E83163B08BC00831200288316682E6C
:101A600083163B08BC0083129B2B8316682E8316BB
:101A70003B08BC00BC080319412D3C08023C031D77
:101A8000A22DDC01DB018A1183122C278A1502307A
:101A90008316DD003F30DF00FF30DE008A11831245
:101AA0001F278A158316BE01BD01BE08031D852DA3
:101AB0003D087F3C031C852D0830E0008A1183120D
:101AC0009E228A1502308316E0008A118312C620F6
:101AD0008A1517308316E0008A1183129E228A1518
:101AE000203083162007BF002108C0000318C00A59
:101AF0004008DC003F08DB008A1183122C278A157E
:101B00008316BD0A0319BE0A552D2030DC00DB0107
:101B10008A1183122C278A1508308316E0008A1157
:101B200083129E228A1502308316E0008A118312E6
:101B3000C6208A1517308316E0008A1183129E2270
:101B40008A1583163C0BA52DA92D3C08023C031DCC
:101B5000E92DDC01DB018A1183122C278A15033061
:101B60008316DD00DF01FF30DE008A1183121F279C
:101B70008A158316BE01BD013E08003C031CE92DF9
:101B80000830E0008A1183129E228A1502308316E3
:101B9000E0008A118312C6208A1517308316E000F0
:101BA0008A1183129E228A15013083162007BF00F6
:101BB0002108C0000318C00A4008DC003F08DB0011
:101BC0008A1183122C278A158316BD0A0319BE0AAF
:101BD000BC2D682E83163B08BC000230BD001730B8
:101BE000BE002030DC00DB018A1183122C278A150D
:101BF00083163C08F700F70883120319042E0130FE
:101C0000770203190F2E1B2E09308316E0008A116C
:101C100083129E228A1508308316BC00212E0B30B9
:101C20008316E0008A1183129E228A1508308316DB
:101C3000BC00212E83121F308316BC000830BD006B
:101C4000BE013C08E0008A1183129E228A15831689
:101C50003D08E0008A118312C6208A158316BE084B
:101C60000319392E3E08E0008A1183129E228A153C
:101C70008316682E83163B08BC008312ED2B831657
:101C8000682E83163B08BC002C08DC002B08DB0008
:101C90008A1183122C278A1502308316DD003F300B
:101CA000DF00FF30DE008A1183121F278A150930FA
:101CB0008316E0008A1183129E228A150A30831649
:101CC000E0008A118312C6208A158316682E8316B7
:101CD00083128A150A12852E0A108A140A158207A1
:101CE000292C8E2C972CAF2C292D302D372DEA2D19
:101CF0003A2E412E2808FF3E0318862E013E8B2ED9
:101D000083163A08BB008312212C862E87110712F6
:101D10008A150A12952E0A108A140A158207802E37
:101D20002A088316BA0083127A2E0730A9000130E0
:101D3000EF008A1169208A158A110A1606292808D7
:101D4000FF3E0318B12E013EB62E83164008C60092
:101D50003F08C5004308C7004408C8008312CD21CE
:101D6000B12E871107128A150A12DC2E0A108A1466
:101D70000A158207A52E8316BD0183122C0883162F
:101D8000BC0083122B088316BB0083122A0883161B
:101D9000BA00043083126F028316BE003D08C200F1
:101DA0003C08C1003B08C0003A08BF002D30C3000A
:101DB0003E08C40083129F2E0730A9000130EF00B7
:101DC0008A1169208A158A110A1610292808FF3EEF
:101DD0000318FA2E013EFF2E83163F08C5003E0869
:101DE000C4004208C6004308C7008A118312D227E4
:101DF0008A15FA2E871107128A150A12262F0A143D
:101E00008A140A158207EC2E8316BD0183122C0852
:101E10008316BC0083122B088316BB0083122A088A
:101E20008316BA0083122D08EF0083163D08C10007
:101E30003C08C0003B08BF003A08BE002D30C2007D
:101E400083126F088316C3008312E62EC430A900E4
:101E50000430EF078A1169208A158A110A161A2997
:101E60002808FF3E03188D2F013E922F83163E084F
:101E7000C2003D08C1003F08C3004008C40042083A
:101E8000DC004108DB008A1183122C278A15831697
:101E9000C5014408450203188B2F450843078400F9
:101EA0000008C6000330DD00DF014608DE008A11AD
:101EB00083121F278A1583162808E0008A118312CF
:101EC0009E228A1583162508E0008A118312C620F7
:101ED0008A1583162608E7008312AE208316A90808
:101EE0000319792F2908E0008A1183129E228A158E
:101EF000831601302007C6002108C7000318C70A4F
:101F00004708DC004608DB008A1183122C278A155B
:101F10008316C50A492F83128D2F871107128A1540
:101F20000A12AD2F0A148A140A158207362F2B08BD
:101F30008316BB0083122A088316BA00033083126B
:101F40006F028316BC003B08BE003A08BD002C306F
:101F5000BF003C08C0008312302F0730A9000130B9
:101F6000EF008A1169208A158A110A162429280887
:101F7000FF3E0318EC2F013EF12F83163D08C100F0
:101F80003C08C0003E08C2003F08C300C40143082B
:101F900044020318EA2F4108FA004008C00A031956
:101FA000C10AC7007A08C800DC004708DB008A11B4
:101FB00083122C278A1505308316D900C530DA0024
:101FC0008312452083164408420784004508800098
:101FD000C40AC72F8312EC2F871107128A110A1621
:101FE00019280A148A140A158207BD2F29080C1E05
:101FF000F72F99002908EE060034FF3FFF3FFF3F0F
:102000002B088316BB0083122A088316BA0083129A
:102010002C08EF0083163B08BD003A08BC002C30AA
:10202000BE0083126F088316BF000A128A1583123E
:10203000B72F0A168A11E230A9000330EF070A12FF
:1020400069200A168A110A162C290A124B200A1630
:10205000D030A900AA01AB01AC01AD010530EF0001
:102060000A1269200A168A110A1632290A127B22DC
:102070000A16D030A9000130AA00AB01AC01AD01B5
:102080000530EF000A1269200A168A110A1638294B
:1020900001308316B900BD012930BE00BD08031D03
:1020A0009E280A12831252200A1678088316BA0054
:1020B0003A08043C031964280A12831252200A16B3
:1020C00078088316BA0058280A12831252200A167A
:1020D0007808EF008316BC00BB0183126F088316DB
:1020E0003B02031885283E08BF000A1283125220C3
:1020F0000A1683163F088400780880003E08840092
:102100000008BC06BE0ABB0A6D280A1283125220C0
:102110000A1678088316BC06031D97280130BD00F7
:10212000063083120C1E922899009C2883160530D5
:1021300083120C1E9928990083164E2883122908B1
:10214000103C031DA7280A12B2200A163C292908B0
:10215000113C031DAF280A12D9280A163C29290868
:10216000123C031DB7280A124D290A163C292908DA
:10217000143C031DBF280A12DE290A163C2929082F
:10218000153C031DC7280A12AA210A163C29290852
:10219000173C031DCF280A12F8290A163C292908E2
:1021A000183C031DD7280A123A2A0A163C29290886
:1021B0001A3C031DDF280A12672A0A163C2929083F
:1021C0001B3C031DE7280A12712A0A163C2929081C
:1021D000413C031DEF280A12542E0A163C292908F7
:1021E000403C031DF7280A12682E0A163C292908CC
:1021F000473C031DFF280A12AE2E0A163C29290867
:10220000433C031D09290A128A15902E0A168A11C9
:102210003C292908423C031D13290A128A15BB2EAA
:102220000A168A113C292908443C031D1D290A125B
:102230008A15042F0A168A113C292908453C031DDA
:1022400027290A128A15972F0A168A113C2929086C
:10225000463C031D2D2900283C292908503C031D1C
:10226000332925283C292908513C031D39293628C2
:102270003C298316B901831283163908F8008312AA
:102280008A150A160B2E8316661464008312071E25
:102290005E29640083166508E503003A031D55298D
:1022A000661083125E295D298316FF30E7000A124B
:1022B0008A158312AE200A168A1147290030831628
:1022C00066180130F8008312003483165D0DDE00BD
:1022D000DE0DDE0DF830DE050716FF30E500831257
:1022E00043218316E001DF0160087102031C862987
:1022F000031D7E295F087002031C86290230F70047
:10230000F70B8029DF0A0319E00A74298312871565
:102310008316E001DF0160087102031C9E29031D82
:1023200095295F087002031C9E290630F700F70B01
:1023300097290000DF0A0319E00A8B298312071A84
:10234000A3290310A42903148316E10DE20DE30D64
:1023500007128312071283165D0BB4290310D90DDF
:10236000031CB4290716C9295D08023C031DBF29B7
:102370000310D90DDA0D031CBF290716C9295D0802
:10238000033C031DC9290310D90DDA0DDB0D031819
:102390000716831287118316E001DF0160087102BE
:1023A000031CE129031DD8295F087002031CE129E1
:1023B0000630F700F70BDA290000DF0A0319E00AFC
:1023C000CE290716DE0B862907166108F70062087A
:1023D000F8006308F9006408FA0083120034040866
:1023E000F8000830F7000718F3298316D501F7170E
:1023F0000B2AF7130B2A03108312071803148316F2
:10240000D50C77170B2A7713F70BFB297808840074
:102410005508F800222A023084000030F71B55309E
:10242000F800F80B112A840B0D2AAB30F71B2E3065
:10243000F800F80B192A00000000F71BF929771B98
:10244000032AFB2983128A110A16212B08300C1E3D
:10245000272A99008316510883120C1E2D2A9900F1
:10246000003407100830F800000000000000F817E2
:102470004A2AF8138316D20C831203180714031C7C
:10248000071078174A2A7813F80B3A2A0000000040
:10249000000007140230F7008401840B4D2AF70B6B
:1024A0004C2AAD308400840B532A00000000F81B36
:1024B000392A781B432A8A110A16AB2BFF30831660
:1024C000CF00D000D100D201E50183124321F808EA
:1024D00003198A2A2808FF3E03188A2A013E952AF2
:1024E0008316DC01DB014030DA00D9010230DD0067
:1024F0008312652178081F39FA007708F8007A08F6
:10250000F9008316D201D1017908D0007808CF00F4
:1025100083128A2A83164F08F7005008F8005108E2
:10252000F9005208FA00831200340A108A140A11C2
:102530008207702AFF308316CB00CC00CD00CE017D
:10254000E50183124321F8080319F52A2808FF3E04
:102550000318F52A013EE42B83164708D0004608ED
:10256000CF004708D2004608D100FF30D300D40086
:102570005108F70052081F39FA005108D5007A08AF
:10258000C038D600D701D8015808DC005708DB0056
:102590005608DA005108D9000230DD0083126521A7
:1025A0008316E50183124321F8080319E82A8316EC
:1025B000DC01DB014030DA00D9010230DD0083129A
:1025C000652177088316D30078081F39D400831259
:1025D00083165308F8005408F900CE01CD0179089C
:1025E000CC007808CB008312F52A8316CA08031999
:1025F000BC2B4F104F18BC2BE50183124321F80868
:102600000319042B8316BC2BD0308316D10052142F
:10261000D21086108312861483160714741C152B8F
:102620005108840001308000482BD218482B6400E8
:1026300083120718292B831651088400D4008312B3
:10264000EF2983165408840078088000D214472BA1
:1026500083120A12F8270A16F80803193B2B0A12EC
:1026600052200A167808023C031D3A2B8316D21416
:1026700052108312462B8316E50183124321F8087A
:102680000319462B8316D214521083128316152B6E
:10269000003052180130F800F8080319B82B500820
:1026A000F7000130770283120319572BB12B013049
:1026B0008316D10083122622D0308316D100521403
:1026C000D210D2189B2BE50183124321F80803197D
:1026D0006B2B83169B2B0A12F8270A16F80803198E
:1026E000992B83165108D3000A12831252200A161E
:1026F000831653088400780880005108840000087D
:10270000083C031D902B5108D3000A12831252205B
:102710000A1683165308840078088000D214982B78
:10272000510884000008023C031D982BD21452105B
:1027300083128316612B003052180130F800F8081C
:102740000319AD2B74105008D100861407105108DE
:10275000D2008312312AB02B831674144F148312C3
:10276000B62B83165008D10083122622BA2B83166B
:102770004F1483128316FA2A4B0FC52B4C0FC52B0F
:102780004D0FC52BCE080319CF2B4B0FDA2B4C0F57
:10279000DA2BCD08031DDA2BCE08031DDA2B8312AA
:1027A0005E227A088316CE007908CD007808CC0026
:1027B0007708CB004B08F7004C08F8004D08F900EB
:1027C0004E08FA00831200340A148A140A11820790
:1027D000AC2A0A124B200A1687150A127B220A1607
:1027E0001030F700F70BF22B00008711FF30831633
:1027F000E500831243218316C901C801C701C60140
:10280000CA0183129A220A124B200A1687150A124D
:102810007B220A161030F700F70B0C2C00008711F2
:102820008316DC01DB014030DA00D9010230DD0023
:102830008312652178081F39FA007708F8007A08B2
:10284000F90000348316C401C5010230F100713073
:10285000F000FF30E50083124321F8080319922CA1
:102860008316DC01DB011030DA00D9010230DD0013
:1028700083126521831607168312071A3D2C8316CF
:10288000C501C40183128715F3010130F200071A54
:10289000522CF20A0319F30A720873040319522C1A
:1028A0006400472C071A5D2CF20A0319F30A720818
:1028B000730403195D2C6400522C8312071E6F2CC5
:1028C0008316C40A0319C50A4408450403196F2C6A
:1028D00012306400FF3E031D692C00005D2C831242
:1028E00087117208730403198C2C8316440845045D
:1028F000031D7C2C83128C2C450CF100440CF00041
:10290000F10CF00CF10CF00CF10CF00CF10CF00CE3
:102910000730F105912C83120230F1007130F00084
:102920008316831283164408F8004508F9008312C1
:102930000034831605118312051583168512831240
:10294000851683168610831286140230F1007130CA
:10295000F0002808FF3E0318BA2C013ED72CE923CB
:10296000E9238316C301C2017908C1007808C000B9
:102970008312BA2C2224FF308316E50083124321F0
:10298000F808031DCA2C8316C301FF30C200C10022
:10299000C000831283164008F7004108F80042087F
:1029A000F9004308FA0083128A110A16052F0A104B
:1029B0008A100A158207AF2C0A108A100A1582079E
:1029C000512F03300C1EE22C99008316410883120C
:1029D0000C1EE82C9900831641088312EE00003487
:1029E0006E080C1EF12C99000A1252200A16780863
:1029F000063C031DF42C0034063C031DF82C003467
:102A000084011F308305073083169F0040309900F2
:102A100026309800903083129800A001A101103058
:102A2000A2003030A3008A30A400A501A6012D30F9
:102A3000A70040308316990026309800903083120A
:102A40009800403083169900263098009030831209
:102A500098004030831699002630980090308312F9
:102A600098000F30F70007308101813084000008A2
:102A7000F0390738800064000008F03977048000DE
:102A800099256400DF26412D63008C1A492D6400CE
:102A9000452D8C1E492D1A088316A0008312981C00
:102AA000572D1A088316A0008312181218168316C1
:102AB0002008F800831200342808073C031D652D08
:102AC00007300C1E612D9900982D0530FC007C0804
:102AD000063C0319982D7C08053C031D942D2830D5
:102AE000FE006E08F60004300C1E742D99006E086E
:102AF0000C1E782D9900FD016E087D020318902DA3
:102B00007E08840000088316A00083120C1E862D08
:102B100099007E0884000008F606FE0AFD0A7C2D56
:102B200076080C1E912D990045257808FC00672D2C
:102B30000034B130A8000130EE005C250034F20111
:102B40002830F300F208031DDA2D45257808EF0040
:102B50006F08043C0319B02D45257808EF00A82D17
:102B600045257808EE006E08F100F0016E0870024D
:102B70000318C82D7308F4004525740884007808EC
:102B80008000730884000008F106F30AF00AB62DED
:102B900045257808F106F108031DD52D0130F20016
:102BA00006300C1ED12D9900D92D05300C1ED62DC6
:102BB0009900A22D00347C0803178D007D088F003A
:102BC00083168C170C140000000083120E08FA0004
:102BD0000C08F8000E08F900031300347D08143CBB
:102BE0000318F62D7D08163C03181F2E7C080317CA
:102BF0008D007D088F0083160313200883120317AE
:102C00008C00831603132108831203178E0083168A
:102C10008C170C15831203130B08F8008B13831603
:102C2000031755308D00AA308D008C140000000071
:102C30008C18182E0C117808831203138B0400349F
:102C40001F30AA052A08F0002908EF006F08033991
:102C5000F400FC30EF05F301740873020318492EE9
:102C60007008FD006F08FC00DB257908F200780889
:102C7000F1007008FD006F08FC0072088316A100C7
:102C80007108A0008312EE25EF0A0319F00AF30A77
:102C90002C2E2B30F5000330F3006E08730203185E
:102CA000812E750884000008F100840A0008F200F3
:102CB000F50AF50AF008031D702E6F08033C031C8B
:102CC000702E03106F0DF900700DFA007908203E88
:102CD0008400840A720880008403710880007B2EBF
:102CE0007008FD006F08FC0072088316A1007108CF
:102CF000A0008312EE25EF0A0319F00A0230F30751
:102D00004D2E6F080339F400F4080319AB2EF008B8
:102D1000031D8E2E6F08033C0318AB2E7408043C71
:102D20000319AB2E7008FD006F08FC00DB25790845
:102D3000F2007808F1007008FD006F08FC007208CE
:102D40008316A1007108A0008312EE25F40AEF0A91
:102D50000319F00A8E2E0730A8000130EE005C2522
:102D60000034EF016F08033C031CCD2E03106F0DE0
:102D7000F700203E8400840A0008F3008403000862
:102D8000F200FD016F08FC0073088316A1007208B1
:102D9000A0008312EE25EF0AB22ECD2E0034E430CF
:102DA000A8002030A9000230EE005C25003428087D
:102DB000A900FF30A8000230EE005C2500349F25FA
:102DC0002808313C031DE62E9925F92E2808323CAF
:102DD000031DEC2E2026F92E2808333C031DF22E6D
:102DE000B126F92E2808193C031DF82ECF26F92EFE
:102DF000D7260034FF3FFF3FFF3FFF3FFF3FFF3F2E
:102E0000BB308316BF008312992C7A088316BE004C
:102E10007908BD007808BC007708BB00D030831269
:102E2000A9008316E50183124321F80803191A2F1C
:102E300000301B2F0130AA0083163F08BF0A840010
:102E400000088312AB0083163F08BF0A8400000805
:102E50008312AC0083163F08840000088312AD0083
:102E60000530EF000A1269200A168A150A16402D4D
:102E70008316C301FF30C200C100C000E501831208
:102E80004321F808031D702F8715A630F700F70BB4
:102E9000472F000087112808FF3E03186B2F013EC3
:102EA000DC2C8316DC01DB014030DA00D901023072
:102EB000DD008312652178081F39FA007708F800D1
:102EC0007A08F9008316C301C2017908C1007808A5
:102ED000C00083126B2FFF308316E500831243215D
:102EE00083164008F7004108F8004208F90043083B
:102EF000FA0083128A110A16822FBB308316BF0094
:102F00008312382F7A088316BE007908BD0078082E
:102F1000BC007708BB00D0308312A9008316E501FE
:102F200083124321F8080319972F0030982F01309E
:102F3000AA0083163F08BF0A840000088312AB0072
:102F400083163F08BF0A840000088312AC00831672
:102F50003F08840000088312AD000530EF000A121C
:102F600069200A168A150A16482DBB308316BF0041
:102F70008A1583126C288A117A088316BE00790894
:102F8000BD007808BC007708BB00D0308312A900D0
:102F90008316E50183124321F8080319D12F00306D
:102FA000D22F0130AA0083163F08BF0A8400000810
:102FB0008312AB0083163F08BF0A84000008831207
:102FC000AC0083163F08840000088312AD00053072
:102FD000EF000A1269200A168A150A16562D2908CA
:102FE000AA00FF30A9000230EF000A1269200A1679
:102FF0008A150A169C2DFF3FFF3FFF3FFF3FFF3F13
:1030000083164014BB30BF0083126F08053C031DBC
:1030100015282D080139003A031D12288316401087
:10302000142883128316401483128316C40183125A
:103030002C088316C30083122B088316C200831248
:103040002A088316C100003040180130C50044082A
:10305000C9004308C8004208C7004108C600450827
:10306000CA008A1183129A228A157A088316BE0032
:103070007908BD007808BC007708BB00D030831207
:10308000A9008316E5018A11831243218A15F808E5
:1030900003194C2800304D280130AA0083163F0840
:1030A000BF0A840000088312AB0083163F08BF0AE2
:1030B000840000088312AC0083163F0884000008D7
:1030C0008312AD000530EF000A128A1169200A163A
:1030D0008A158A150A164F2DFF308316E5008A11CE
:1030E000831243218A15F8080319A4282808FF3EF3
:1030F0000318A428013EC2288316DC01DB01FF303F
:10310000DA00D9000230DD008A11831265218A15A8
:103110008316DC01DB014030DA00D9010230DD002A
:103120008A11831265218A1578081F39FA007708F9
:10313000F8007A08F9008316C301C2017908C100BA
:103140007808C0008312A428FF308316E5008A1196
:10315000831243218A15F808031DB5288316C3017D
:10316000FF30C200C100C000831283164008F70080
:103170004108F8004208F9004308FA0083128A1156
:103180000A16BB2F0A108A100A1182077C28BB304E
:103190008316BF008A1183125E228A157A0883166D
:1031A000BE007908BD007808BC007708BB00D030AD
:1031B0008312A9008316E5018A11831243218A151F
:1031C000F8080319E5280030E6280130AA00831624
:1031D0003F08BF0A840000088312AB0083163F0833
:1031E000BF0A840000088312AC0083163F088400E5
:1031F00000088312AD000530EF000A128A11692021
:103200000A168A158A150A165D2D8316C401FF3029
:10321000E5008A11831243218A15F80803191F2932
:103220008316DC01DB01DA01D9010130DD008A11EE
:10323000831265218A1577088316C40083128316CA
:103240004408F8008312003429308316BD0083122D
:103250002B088316BC0083122A088316BB00831236
:103260002C088316BF0003303F07C000C1008A113D
:103270008312E1248A1583163D088400E030800023
:103280000A128312F6270A1683163D088400831259
:103290002A0880000A12F6270A1683163D088400C1
:1032A00083122B0880000A12F6270A1683163D089F
:1032B000C0003C08C2003B08C100FF30E5008A1195
:1032C000831243218A15F8080319862983164108B9
:1032D000F70042080F39FA004108C4007A08403864
:1032E000C500C601C7014708DC004608DB004508E9
:1032F000DA004108D9000230DD008A11831265210D
:103300008A15052178088316C3008312FF308316BF
:10331000E5008A11831243218A15F808031D9429B8
:10332000FF308316C300831283164308F800400859
:103330008400780880000A128312F6270A160130EA
:103340008316BE003F083E020318B6293D08C000A0
:1033500083120521831640088400780880000A1231
:103360008312F6270A168316BE0AA2298A1183122F
:10337000F0248A158A150A16632D2B088316BD00C2
:1033800083122A088316BC000330BB0083126F0827
:1033900083163B020318232A3D08FA003C08BC0AA6
:1033A0000319BD0ABE007A08BF0029303B0784001C
:1033B0000008C0003F08C2003E08C1004008C3002A
:1033C000FF30E5008A11831243218A15F80803199A
:1033D000202A83164108F70042080F39FA004108F5
:1033E000C4007A085038C500C601C7014708DC0090
:1033F0004608DB004508DA004108D9000230DD004C
:103400008A11831265218A15FF308316E5008A111F
:10341000831243218A1583164308C4006030C50017
:10342000C601C7014708DC004608DB004508DA0092
:103430004308D9000230DD008A11831265218A1504
:103440008316BB0AC62907308312A9000130EF009A
:103450000A128A1169200A168A158A150A16692D18
:1034600083164708C8002030C900CA01CB014B08A9
:10347000DC004A08DB004908DA004708D9000230BE
:10348000DD008A11831265218A158316DC01DB01B8
:103490004030DA00D9010230DD008A118312652143
:1034A0008A1578088316CA007708C9004A08FA0105
:1034B000F800831200348316C501FF30E5008A113D
:1034C000831243218A15F8080319762A2808FF3E3B
:1034D0000318762A013E7D2A83164308C70083120B
:1034E000302278088316C5008312762A8316450891
:1034F000F80083128A150A16CA2A0A108A140A11B9
:1035000082076C2A29308316BD0083122B0883168C
:10351000BC0083122A088316BB0083122C08831672
:10352000BF0003303F07C000C1008A118312E124AD
:103530008A1583163D088400E23080000A12831247
:10354000F6270A1683163D08840083122A08800095
:103550000A12F6270A1683163D08840083122B08E8
:1035600080000A12F6270A168316BE013F083E02A3
:103570000318D62A3D08C0003C08FA003B08BB0AE5
:103580000319BC0AC1007A08C200C4004108C30084
:1035900083125B2A831640088400780880000A1290
:1035A0008312F6270A168316BE0AB62A8A118312D8
:1035B000F0248A158A150A166F2DFF308316E50050
:1035C0008A11831243218A15F8080319292B280828
:1035D000FF3E0318292B013E2C2B83163E08C20008
:1035E0004008C3004108C400C5014408450203184F
:1035F000272B45084207C600C700831230228316D6
:103600004308450784000008C600C700FF30E500F6
:103610008A11831243218A15F8080319242B831673
:103620004708C8003030C900CA01CB014B08DC0094
:103630004A08DB004908DA004708D9000230DD00FB
:103640008A11831265218A158316C50AF52A831209
:10365000292B8A150A16472B0A148A140A11820785
:10366000ED2A2B088316BC0083122A088316BB00A0
:10367000033083126F028316BD003C08BF003B0875
:10368000BE002C30C0003D08C1008312DD2A073087
:10369000A9000130EF000A128A1169200A168A1562
:1036A0008A150A16752DFF308316E5008A118312DC
:1036B00043218A15F8080319AF2B2808FF3E031889
:1036C000AF2B013EB22B83164108C7004008C6004D
:1036D0004408C8004508C9004608CB004708CC008C
:1036E0000830CD00CE014E08DC004D08DB00470855
:1036F000DA004608D9000330DD008A118312652103
:103700008A158316DC010930DB00DA01D9010330A8
:10371000DD008A11831265218A158316CA014908C2
:103720004A020318AD2B4808C80AC80ACB00DC01BE
:103730000930DB00DA01D9010330DD008A11831280
:1037400065218A1583164B08840077088000840A57
:10375000780880000230CA078F2B8312AF2B8A159E
:103760000A16D92B0A148A140A118207632B8316AE
:10377000BF0183122C088316BE0083122B08831608
:10378000BD0083122A088316BC0083122D08EF00A7
:1037900083163F08C3003E08C2003D08C1003C0834
:1037A000C0002D30C40083126F088316C500831239
:1037B000532BC430A9000430EF070A128A11692084
:1037C0000A168A158A150A167B2DFF308316E50026
:1037D0008A11831243218A15F80803193C2C280802
:1037E000FF3E03183C2C013E3F2C83164208C800C4
:1037F0004108C7004508C9004608CA004708CC0070
:103800004808CD000830CE00CF014F08DC004E083C
:10381000DB004808DA004708D9000330DD008A11D0
:10382000831265218A158316CB014A084B020318BF
:103830003A2C4908C90AC90A8400840A0008FA0017
:1038400084030008CC007A08CD000A30CE00CF01F6
:103850004F08DC004E08DB004D08DA004C08D900A8
:103860000330DD008A11831265218A150230831628
:10387000CB07152C83123C2C8A150A16652C0A10CE
:103880008A100A158207F52B8316BF0183122C08B4
:103890008316BE0083122B088316BD0083122A08EC
:1038A0008316BC00043083126F028316C0003F08E9
:1038B000C4003E08C3003D08C2003C08C1002D30D2
:1038C000C5004008C6008312E52B0730A90001306F
:1038D000EF000A128A1169200A168A158A150A163B
:1038E000812D2A308316BB0097308312A9008316DE
:1038F0003B08BC008A11831222248A1583163C08D7
:103900008400840A790880008403780880000330EA
:103910008312EF000A128A1169200A168A158A1585
:103920000A16872D2A308316BB0083122C08EF005D
:1039300083163B088400840A0008BD008403000845
:10394000BC003D08BF003C08BE002C30C000831204
:103950006F088316C100E6308312A9000330EF0719
:103960000A128A1169200A168A158A150A168D2DDF
:103970002A308316BB003B088400840A0008BD007F
:1039800084030008BC00033083126F028316BE005C
:103990003D08C0003C08BF002C30C1003E08C200FA
:1039A00007308312A9000130EF000A128A11692042
:1039B0000A168A158A150A16932D8316BB013B0831
:1039C000033C031C2F2DBD013B08BC0003103B0D25
:1039D000F700BE003E0A0A128A11831235200A1629
:1039E0008A15FA0083163E080A128A1183123520BE
:1039F0000A168A158316BF007A08C0003C08831295
:103A000003178D00831603133D08831203178F00DD
:103A1000831603133F08831203178C0083160313C6
:103A20004008831203178E0083168C170C1583121F
:103A300003130B08F8008B138316031755308D0002
:103A4000AA308D008C14000000008C18252D0C115C
:103A50007808831203138B048316BB0ADF2C8A01B8
:103A6000831282018A150A16992D8316BA08031D3E
:103A70009E2D83122908523C031D422D8A11002FCE
:103A80008A159D2D2908533C031D4A2D8A117D2F2F
:103A90008A159D2D2908543C031D502D00289D2D6D
:103AA0002908553C031D582D8A11B52F8A159D2DC7
:103AB0002908563C031D5E2DC7289D2D2908603C12
:103AC000031D642D24299D2D2908613C031D6A2DA9
:103AD000BD299D2D2908623C031D702D822A9D2D34
:103AE0002908633C031D762D312B9D2D2908653C4B
:103AF000031D7C2DB72B9D2D2908643C031D822DB1
:103B0000442C9D2D2908663C031D882D712C9D2D6C
:103B10002908673C031D8E2D922C9D2D2908683C99
:103B2000031D942DB82C9D2D2908313C031D9A2D81
:103B3000DD2C9D2D8A11EF2F8A15831683128A158D
:103B40000A16122E84011F308305073083169F004A
:103B50004030990026309800903083129800403011
:103B600083169900263098009030831298004030D8
:103B700083169900263098009030831298004030C8
:103B800083169900263098009030831298004030B8
:103B90008316990026309800903083129800713077
:103BA000F0000230F10074100714071499308316E6
:103BB0008700103086000B308500B53083129000EE
:103BC0008F018E0183160C14C03083128B040F30CA
:103BD000F70007308101813084000008F039073890
:103BE000800064000008F039770480000A128A110E
:103BF0004B200A168A150A128A11B2200A168A1553
:103C00000B138B138B1B012E83160C1083120615BE
:103C100064008A1148288A1578088316B900BA000A
:103C20008312352D082E6300FF3FFF3FFF3FFF3F0C
:103C3000FF3FFF3FFF3FFF3FFF3FFF3FFF3FFF3F94
:103C4000FF3FFF3FFF3FFF3FFF3FFF3FFF3FFF3F84
:103C5000FF3FFF3FFF3FFF3FFF3FFF3FFF3FFF3F74
:103C6000FF3FFF3FFF3FFF3FFF3FFF3FFF3FFF3F64
:104200002000FF00FF00FF00FF00FF00FF00FF0095
:10421000FF00FF00FF00FF00FF00FF00FF00FF00A6
:10422000FF00FF00FF00FF00FF00FF00FF00FF0096
:10423000FF00FF00FF00FF00FF00FF00FF00FF0086
:10424000FF00FF00FF00FF00FF00FF00FF00FF0076
:10425000FF00FF00FF00FF00FF00FF00FF00FF0066
:10426000FF00FF00FF00FF00FF00FF00FF00FF0056
:10427000FF00FF00FF00FF00FF00FF00FF00FF0046
:10428000FF00FF00FF00FF00FF00FF00FF00FF0036
:10429000FF00FF00FF00FF00FF00FF00FF00FF0026
:1042A000FF00FF00FF00FF00FF00FF00FF00FF0016
:1042B000FF00FF00FF00FF00FF00FF00FF00FF0006
:1042C000FF00FF00FF00FF00FF00FF00FF00FF00F6
:1042D000FF00FF00FF00FF00FF00FF00FF00FF00E6
:1042E000FF00FF00FF00FF00FF00FF00FF00FF00D6
:1042F000FF00FF00FF00FF00FF00FF00FF00FF00C6
:10430000FF00FF00FF00FF00FF00FF00FF00FF00B5
:10431000FF00FF00FF00FF00FF00FF00FF00FF00A5
:10432000FF00FF00FF00FF00FF00FF00FF00FF0095
:10433000FF00FF00FF00FF00FF00FF00FF00FF0085
:10434000FF00FF00FF00FF00FF00FF00FF00FF0075
:10435000FF00FF00FF00FF00FF00FF00FF00FF0065
:10436000FF00FF00FF00FF00FF00FF00FF00FF0055
:10437000FF00FF00FF00FF00FF00FF00FF00FF0045
:10438000FF00FF00FF00FF00FF00FF00FF00FF0035
:10439000FF00FF00FF00FF00FF00FF00FF00FF0025
:1043A000FF00FF00FF00FF00FF00FF00FF00FF0015
:1043B000FF00FF00FF00FF00FF00FF00FF00FF0005
:1043C000FF00FF00FF00FF00FF00FF00FF00FF00F5
:1043D000FF00FF00FF00FF00FF00FF00FF00FF00E5
:1043E000FF00FF00FF00FF00FF00FF00FF00FF00D5
:1043F000FF00FF00FF00FF00FF00FF00FF00FF00C5
:08400000FF3FFF3FFF3FFF3FC0
:00000001FF
